:10000000831602309F0089018601BF3087002430AB
:100010009800813099008312903098000730890051
:100020008317A03084000830A600FF3086007020BF
:10003000003086008C1E1A28181951289818592843
:100040001A088000840AA60B1A2800308000A0300D
:1000500084000930A6000008A50026084620A70055
:10006000A50C031C42284428091100000915A70B00
:100070003028840AA60B2B288914000009100000E0
:1000800009141028891034288914342882070000A4
:1000900002340434043404340434043404340434A2
:1000A00003340F3086007020003086001A08981C38
:1000B0001028F030860070200030860018121816C4
:1000C0001028A530A00000000000A00B6528080043
:1000D0006330A100000000006120A10B6C28080023
:1000E0006330A2006230A3000330A4000000682047
:1000F000A20B77286120A30B7A28A40B7D28080087
:00000001FF
